:1000000000308A007C290000283084000008031991
:1000100018280130A100A001A00B0C28A10B0B286F
:100020004A30A000A00B122800000000800B092815
:10003000003429308400FC308005800C800C0008DE
:100040000319262824280000800B23280034A70148
:100050002708273C031C3F28831605128312051628
:10006000EF30A000A00B322800000000831605121C
:10007000831205121430A8000420A70A2828A7011B
:100080002708273C031C5B288316051283120516DC
:100090000130A80004200230A800AB30A9001920CC
:1000A000A80B4D2883160512831205121430A800E0
:1000B0000420A70A4028A7012708273C031C77280B
:1000C00083160512831205160230A80004200230A0
:1000D000A8007930A9001920A80B692883160512F9
:1000E000831205121430A8000420A70A5C28A70177
:1000F0002708273C031C9328831605128312051634
:100100000130A80004200230A800AB30A90019205B
:10011000A80B852883160512831205121430A80037
:100120000420A70A78282728952983160513831207
:10013000051383168513831285170630A700FA303E
:10014000A8000420A70B9F2883160513831205130C
:1001500083168513831285130230A7009630A800FA
:100160000420A70BAE2883160513831205178316E8
:100170008513831285130630A700FA30A8000420E7
:10018000A70BBD28952897298316051083120514FF
:1001900083168510831285148316051183120515A5
:1001A0008316851183128515831605108312051495
:1001B0008316851083128514831605118312051585
:1001C0008316851183128515A7012708193C031C86
:1001D00027298316051083120510831685118312B3
:1001E00085110A30A8000420831685118312851515
:1001F0000A30A800042083168510831285100A3067
:10020000A800042083160510831205140A30A800E4
:10021000042083160511831205110A30A80004205A
:1002200083168510831285140A30A80004208316D3
:100230008511831285110A30A80004208316051148
:10024000831205150A30A8000420A70AE5288316A2
:1002500005108312051483168510831285148316E6
:100260000511831205158316851183128515A701C3
:100270002708193C031C7A298316851183128511DE
:100280000A30A800042083160511831205110A30D4
:10029000A800042083168511831285150A30A80052
:1002A000042083168510831285100A30A8000420CC
:1002B00083160511831205150A30A8000420831641
:1002C0000510831205100A30A8000420831685103B
:1002D000831285140A30A800042083168511831226
:1002E00085110A30A8000420831605108312051416
:1002F000A70A3829D428992984011F30830507309B
:100300009F0000308316850083128501FF3083161D
:10031000860083120608A6000330A6052608FC3EC8
:1003200003189B29043E9C2927289B2995289B2953
:10033000C4289B299B2963000A148A100A1182078A
:080340009429962998299A29B5
:02400E00383F39
:00000001FF
